:020000040000FA
:1000000000020400000000000A1700000A170000A8
:100010000A1700000A1700000A1700000A1700005C
:100020000A1700000A1700000A1700000A1700004C
:100030000A1700000A1700000A1700000A1700003C
:100040000A1700000A1700000A1700000A1700002C
:100050000A1700000A1700000A1700000A1700001C
:100060000A1700000A1700000A1700000A1700000C
:100070000A1700000A1700000A1700000A170000FC
:100080000A1700000A1700000A1700000A170000EC
:100090000A1700000A1700000A1700000A170000DC
:1000A0000A1700000A1700000A1700000A170000CC
:1000B0000A1700000A1700000A1700000A170000BC
:1000C0000A1700000A1700000A1700000A170000AC
:1000D0000A1700000A1700000A1700000A1700009C
:1000E0000A1700000A1700000A1700000A1700008C
:1000F0000A1700000A1700000A1700000A1700007C
:100100000A1700000A1700000A1700000A1700006B
:100110000A1700000A1700000A1700000A1700005B
:100120000A1700000A1700000A1700000A1700004B
:100130000A1700000A1700000A1700000A1700003B
:100140000A1700000A1700000A1700000A1700002B
:100150000A1700000A1700000A1700000A1700001B
:100160000A1700000A1700000A1700000A1700000B
:100170000A1700000A1700000A1700000A170000FB
:100180000A1700000A1700000A1700000A170000EB
:100190000A1700000A1700000A1700000A170000DB
:1001A0000A1700000A1700000A1700000A170000CB
:1001B0000A1700000A1700000A1700000A170000BB
:1001C0000A1700000A1700000A1700000A170000AB
:1001D0000A1700000A1700000A1700000A1700009B
:1001E0000A1700000A1700000A1700000A1700008B
:1001F0000A1700000A1700000A1700000A1700007B
:10020000FFFFFF00FFFFFF000A1700000A170000B2
:100210000A1700000A1700000A1700000A1700005A
:100220000A1700000A1700000A1700000A1700004A
:100230000A1700000A1700000A1700000A1700003A
:100240000A1700000A1700000A1700000A1700002A
:100250000A1700000A1700000A1700000A1700001A
:100260000A1700000A1700000A1700000A1700000A
:100270000A1700000A1700000A1700000A170000FA
:100280000A1700000A1700000A1700000A170000EA
:100290000A1700000A1700000A1700000A170000DA
:1002A0000A1700000A1700000A1700000A170000CA
:1002B0000A1700000A1700000A1700000A170000BA
:1002C0000A1700000A1700000A1700000A170000AA
:1002D0000A1700000A1700000A1700000A1700009A
:1002E0000A1700000A1700000A1700000A1700008A
:1002F0000A1700000A1700000A1700000A1700007A
:100300000A1700000A1700000A1700000A17000069
:100310000A1700000A1700000A1700000A17000059
:100320000A1700000A1700000A1700000A17000049
:100330000A1700000A1700000A1700000A17000039
:100340000A1700000A1700000A1700000A17000029
:100350000A1700000A1700000A1700000A17000019
:100360000A1700000A1700000A1700000A17000009
:100370000A1700000A1700000A1700000A170000F9
:100380000A1700000A1700000A1700000A170000E9
:100390000A1700000A1700000A1700000A170000D9
:1003A0000A1700000A1700000A1700000A170000C9
:1003B0000A1700000A1700000A1700000A170000B9
:1003C0000A1700000A1700000A1700000A170000A9
:1003D0000A1700000A1700000A1700000A17000099
:1003E0000A1700000A1700000A1700000A17000089
:1003F0000A1700000A1700000A1700000A17000079
:10040000EF832100007F220000018800000000002F
:100410000C000700006C2100010020001100070003
:10042000000020000000E000020032000000020096
:1004300000000000F4160200000000000040DA0096
:100440000000FE004440A900000020000000E00081
:100450000300320000002000A00188004440A800F2
:100460000000060091018800800078000000EB0089
:1004700015003700E280400032A0B4009101BA00BC
:10048000E280400032A0B4009102BA00E280400055
:1004900032A0B4000002EB00472BDE00F507B200EB
:1004A000602CE10004003A000059EB008301E900F0
:1004B000FDFF3E00040037006128E100010032002A
:1004C0000082EB00040007001101BA000200E00006
:1004D000E8FF3A00000006003159BA008301E90044
:1004E0000C0032002159BA008301E90008003200F3
:1004F0000400E00003003A00E280400032A0B400B3
:10050000F5FF370011D9BA008301E900FAFF3A007C
:100510008100E800E180400032A0B4000000060045
:1005200000000000000000000000000000000000CB
:1005300000000000000000000000000000000000BB
:1005400000000000000000000000000000000000AB
:10055000000000000000000000000000000000009B
:10056000000000000000000000000000000000008B
:10057000000000000000000000000000000000007B
:10058000000000000000000000000000000000006B
:10059000000000000000000000000000000000005B
:1005A000000000000000000000000000000000004B
:1005B0000200FA00000F78009E0078000040EB0077
:1005C000804878009E0078000040EB009040980042
:1005D0001E0178006000B800100198002101980009
:1005E0009E0078000000EB00B00098009E007800AC
:1005F0000040EB00B04898009E0078000040EB00FF
:10060000804898009E00780010C0B3009048980081
:100610009E00780010C0B300A04898001E0178002A
:100620006000B80000099800110998009E00780049
:100630000000EB00A00898001E0178006000B800E0
:1006400060019800710198000000EB000080FA0042
:10065000000006000200FA00000F78000080FA0097
:10066000000006000800FA00008FBE0072002000A3
:10067000030020003E004100AE80490020079800A2
:10068000310798002E009000BE009000E00F50004F
:10069000E08F580006003D002E019000BE01900042
:1006A00067014100E0814900220798003307980064
:1006B0002E019000BE0190004D1ADD004310DE00B7
:1006C00000007200C398DE000080FA0000000600FF
:1006D0000200FA00000F78009E0078001000200051
:1006E000A70807008000EB000000EB00A40807004B
:1006F000110020000000EB00A10807000080FA00B4
:10070000000006000C00FA002007980061479800DE
:100710000000EB00000F78006E4090000004E00045
:1007200015003A0010002000E9FF07000000EB0070
:1007300010079800090037008000EB000000EB0074
:100740008F080700110020000000EB008C08070054
:100750001E0090000000E800100798001E009000A6
:10076000E40F5000F4FF3400AE0090000040EB00B6
:1007700080487800080137002E00900090407800F3
:100780006E40900080CF5000110032006E4090000B
:10079000E74F500004003A002E009000104078000F
:1007A000E64F500007003A006E409000EE4F5000B8
:1007B00007003A002E00900010407800ED4F5000E6
:1007C0000300320050002000000F7800F2003700D4
:1007D0002E009000904078006E40900080CF500036
:1007E000E8003A006E409000E64F500006003A00E4
:1007F00010002000B6FF0700AE00900070C0B300EC
:1008000080487800DF0037006E409000ED4F5000C8
:10081000DC003A0010002000ADFF0700AE009000A1
:10082000E0C0B30080487800D60037002E0090006A
:10083000104078000080FB006101B9004207980079
:1008400053079800F0002000010020004E019000A6
:10085000DE019000800F5100818F5900C4003E00DE
:100860004E009000DE009000006001000F00370095
:100870001400370019003700270037003500370013
:100880003A003700480037004D0037005B00370062
:10089000690037006E0037007C00370081003700A8
:1008A0008F00370094003700A20037000000EB00F3
:1008B00087FF0700AE00900010C0B30080487800AA
:1008C000B00037001000200081FF0700AE0090004C
:1008D00020C0B30080487800AA0037006E40900026
:1008E000E84F5000060036001000200078FF070097
:1008F000AE00900090C0B30080487800A10037009F
:100900000000EB0072FF0700AE00900030C0B300A3
:10091000804878009B0037006E409000E44F500004
:1009200006003A000000EB0069FF0700AE009000EF
:1009300040C0B300804878009200370010002000CB
:1009400063FF0700AE00900050C0B30080487800FD
:100950008C003700100020005DFF0700AE00900003
:1009600050C0B30080487800860037006E40900089
:10097000E64F500006003A000000EB0054FF07006D
:10098000AE00900060C0B300804878007D00370062
:10099000100020004EFF0700AE00900080C0B300A2
:1009A00080487800770037001000200048FF0700DB
:1009B000AE00900070C0B30080487800710037002E
:1009C0006E409000E44F500006003A000000EB003B
:1009D0003FFF0700AE00900040C0B30080487800A1
:1009E000680037001000200039FF0700AE009000BB
:1009F00080C0B30080487800620037006E409000ED
:100A0000E14F500006003A000000EB0030FF070005
:100A1000AE00900010C0B300804878005900370045
:100A2000100020002AFF0700AE00900020C0B30095
:100A300080487800530037000000EB0024FF0700D7
:100A4000AE009000A0C0B300804878004D00370091
:100A50006E409000EB4F500006003A000000EB00A3
:100A60001BFF0700AE009000B0C0B30080487800C4
:100A7000440037001000200015FF0700AE00900072
:100A8000C0C0B300804878003E003700100020004E
:100A90000FFF0700AE009000C0C0B3008048780090
:100AA000380037006E409000ED4F500006003A00CD
:100AB0000000EB0006FF0700AE009000D0C0B300BE
:100AC000804878002F0037001000200000FF07004A
:100AD000AE009000F0C0B3008048780029003700D5
:100AE00010002000FAFE0700AE009000E0C0B30046
:100AF00080487800230037006E409000EB4F500094
:100B000006003A000000EB00F1FE0700AE00900086
:100B1000B0C0B300804878001A00370010002000F1
:100B2000EBFE0700AE009000F0C0B30080487800F4
:100B3000140037006E409000E14F500006003A006C
:100B40000000EB00E2FE0700AE00900010C0B30012
:100B5000804878000B00370010002000DCFE070002
:100B6000AE00900020C0B300804878000500370038
:100B700050002000000F78002E009000EE40900002
:100B8000014878002E009000904078006E40900060
:100B900080CF500025FF3A001E0078000080FA0048
:100BA000000006001400FA00500798006107980042
:100BB00072079800030F9800140F98000000EB00D4
:100BC000300798000E0890000000E0000A00320094
:100BD0007E009000900078000E08900001087800D8
:100BE0000E0890008080E8007E00900010007800E1
:100BF00000804000300798007E0090008080E80070
:100C00007E009000100078000080400040079800AF
:100C10004A0037004E0090000000E90040079800AD
:100C20004E00900090407800414798000040EB0053
:100C3000304798000000EB00000F78002E003700CE
:100C40005E009000EE00900061005000E0805800CF
:100C500050079800610798001E0890000000E0000F
:100C6000080032005E009000EE009000E00F50009F
:100C7000E08F580003003A0011002000100020000F
:100C80003F0707004E4090000080FB00E10060003D
:100C9000200020003A0707004E4090000080FB0033
:100CA0000000D100404798008000EB000000EB00FE
:100CB000330707003E0090000000E0000A00320009
:100CC00094070700204798002E4090008080FB008A
:100CD0001E0078000008DD00804078003E40900053
:100CE00000C0700030479800110020000000EB00A9
:100CF000230707001E0FE8005E009000EE00900042
:100D0000E00F5000E08F5800030032007000200018
:100D10009E0F1000CAFF34003E0090000000E0006B
:100D2000060032003E0090000000E9003007980005
:100D30003E009000BE409000014878005E009000A8
:100D4000EE009000E00F5000E08F5800B1FF3A0035
:100D50000080FA00000006001C00FA00400798001E
:100D6000214F98006207980073079800040F9800BD
:100D7000150F9800260F9800370F98000000EB0021
:100D8000300798000000EB00200798000040EB00BF
:100D9000204798000000EB00500F9800AE489000EC
:100DA0000EF8970080CF500002003200140020009F
:100DB000540F98005E089000000F78006E009000BD
:100DC000FE009000E00F5000E08F58000C003A0049
:100DD0002EB89700BEB89700E00F5000E08F580083
:100DE0006300320011C0B3004E00900045FE0700C2
:100DF0002EB89700BEB897004D0707005C0037007B
:100E0000AE4890004E0090003EFE07001E027800A3
:100E10009E0990000E0990006E009000FE00900068
:100E200060FF07002E0890000000E0000B00320079
:100E30003E0990009E0890002E08900014060700BE
:100E4000800078000000EB00200798000100E0001F
:100E500002003A0010002000200798001E00E00069
:100E6000320032004E009000104078008040E800D0
:100E70004E009000014878002E0090000000E00035
:100E80001C0032002EB89700BEB89700E00F50004B
:100E9000E08F580017003200AE4090002EF097000F
:100EA00080CF50001300310061C0B3004E009000AD
:100EB00014FE070041C0B3004E00900011FE070071
:100EC0002EB89700BEB89700C289DE004E0ADD003A
:100ED0004201DE00020172002EB89700BEB89700F2
:100EE000000041008180490020BF9F0031BF9F006A
:100EF000030037008EF897004E00900001FE0700B7
:100F00002EB89700BEB89700E00F5000E08F580051
:100F10000600320011C0B3004E009000F9FD07003A
:100F20002EB89700BEB89700010707002E0090006A
:100F30000000E0000E0032000040EB00005F98006F
:100F4000AE4090002EF0970080CF5000020031009C
:100F500014C0B300045F98002E4090000040E800E9
:100F6000204798000E5890000004E000A4FF3A00CB
:100F70002E0090000000E0000C0032002EF09700E0
:100F80000004E00007003200AE4090002EF0970011
:100F900080CF50000300360030002000300798005A
:100FA0000200370020002000300798003E0090002B
:100FB0000080FA00000006001000FA00000F780020
:100FC00012079800230798003107980044079800FB
:100FD000550798006607980077079800BE009000B4
:100FE0004E009000490607006E0090000000E000EF
:100FF00003003200BE0090006E0090004306070020
:101000008F87E8002EF09700E0FF9F002EB8970032
:10101000BEB89700809FBE008F87E8008EF89700CB
:10102000E1FF9F00FE0390006E039000DE0290003F
:101030004E0290001E019000AE01900041C0B3002E
:101040001E00780044FF0700E88757000080FA0080
:10105000000006001200FA0050079800610798008F
:1010600072079800030F98007E019000DE00900048
:101070005E009000EE0507000040EB00304798004E
:101080000040EB00204798006E009000100F7800A1
:101090000E089000100078000000E900400798005A
:1010A000480037004E0090008E0890000080E80055
:1010B0000100400090407800414798004E40900069
:1010C0000004E0003C0032004E009000DE00900082
:1010D0000080E800010040009040780061479800DF
:1010E00010C0B300504798002A0037004E409000CF
:1010F0000080FB00610060000004E0001E00320080
:101100002E4090000004E00009003A001E0FE900A4
:101110001E007800EE0090000080E8000100400012
:10112000904078003147980010C0B30020479800E5
:101130003E409000AE409000014060000004E0009E
:10114000050032006E409000DE40900001407000CB
:1011500060479800050037005E40900080C0EA00BC
:101160006E40900000C06000604798002E409000E4
:1011700000404000204798005E4090000040400042
:10118000504798004E4090000080FB000000D100C6
:10119000404798004E4090000004E000D3FF3A0022
:1011A0004E009000DE0090000080E800010040004A
:1011B000EE409000014878004E0090000000E900E9
:1011C000400798004E0090000000E000B5FF3D0091
:1011D0000080FA00000006000200FA00000F78000C
:1011E0009E00780040002000B00098001E007800AB
:1011F000300090000080FA00000006000200FA00B3
:10120000000F78009E00780010C0B300804878007E
:101210000000EB000080FA00000006000200FA0067
:10122000000F78001E007800A0089000820B2000BC
:101230001E004100B50507000000EB000080FA0029
:10124000000006000800FA00889FBE008A1F780090
:101250003007980064004700F30507004E409000F7
:101260000080FB0001002000FEFC07001007980032
:101270009E00900020032000808F50000300340067
:1012800060002000000F7800230037004E409000DF
:101290000080FB0001002000F2FC070080007800C5
:1012A0003E00900076004000980507003E00900048
:1012B00060019000F00190003E0090009048900086
:1012C0003E009000760240004E4090000084FB00FB
:1012D000090020003E009000680540008F87E8006C
:1012E0000040EB00E0FF9F00829FBE008F87E80078
:1012F000E1FF9F008003EB000003EB008002EB00A6
:101300000801BE00B1C0B3000A00780092FE0700D9
:10131000E8875700000F78001E00E000030032004D
:101320003E0090009E007800310098001E0078007A
:101330004F0578004F04BE000080FA000000060050
:101340000A00FA00881F7800400798004E009000BD
:1013500076004000210020006C0507004E00900040
:101360007600400097040700200798003107980096
:101370002E009000BE009000BAFC070010079800F5
:101380009E00900020032000808F50000300340056
:1013900060002000000F7800200037002E00900031
:1013A000BE009000AFFC0700800078004E00900067
:1013B00076004000550507004E0090006001900047
:1013C000F00190004E009000904890004E00900078
:1013D000760240004E009000680440008F87E800CD
:1013E0000040EB00E0FF9F00829FBE008F87E80077
:1013F000E1FF9F008003EB000003EB008002EB00A5
:101400002E019000BE019000B1C0B300080078002A
:1014100051FE0700E8875700000F78001E00E0002B
:10142000030032004E0090009E00780031009800CA
:101430001E0078004F0478000080FA0000000600CB
:101440000400FA00889FBE008A9FBE001007980023
:101450001E009000A00890001E0090007600400042
:101460002A0507001E009000B04890001E00900062
:1014700060019000F00190001E009000204A900052
:101480001E009000870B2000808343001E00900008
:10149000C5042000808242001E0090002A0820001F
:1014A000000545001E009000F60540001E0090005B
:1014B000000C9000900C90001E009000680040000E
:1014C0008F87E800E1FF9F00829FBE008F87E800C2
:1014D000E4FF9F00050378008A0278000B02780081
:1014E0000801BE0041C0B3001BFE0700E88757009B
:1014F000000F78001E00E000030032001E00900084
:101500009E007800310098001E0078004F05BE0054
:101510004F04BE000080FA00000006000200FA003E
:10152000000F78009E007800768040004100200087
:10153000F60407009E007800768040002104070032
:101540001E01780060019800710198000000EB0016
:101550000080FA00000006000200FA00000F780088
:101560009E0078006B8040002F0507000000EB0014
:101570000080FA00000006000400FA00100798003E
:101580000000EB00000F78001E0090007600400085
:1015900041002000DD0407001E009000760040009E
:1015A000080407001E019000000998001109980026
:1015B0001E009000900890000008900029FC070091
:1015C000800078001E009000210898001E00900006
:1015D000A008900020032000808F500005003400F8
:1015E00060002000000F78001E0090009E00780030
:1015F000310098001E0078000080FA00000006000C
:101600000400FA00889FBE008A9FBE008C1F7800ED
:10161000100798001E009000B04890001E00900037
:1016200060019000F00190001E009000204A9000A0
:101630001E009000870B2000808343001E00900056
:10164000C5042000808242001E0090002A0820006D
:10165000000545001E009000F60540001E009000A9
:10166000200E90001E009000000C9000900C900046
:101670001E009000680040008F87E800E1FF9F0097
:10168000829FBE008F87E800E4FF9F00050378007B
:101690008A0278000B0278008C0078000801BE00F6
:1016A00045FE0700E8875700000F78001E00E000A5
:1016B000030032001E0090009E0078003100980068
:1016C0001E0078004F0678004F05BE004F04BE0094
:1016D0000080FA00000006000200FA00000F780007
:1016E0001E007800A0089000E20E20001E004100BD
:1016F000860407001E007800A00890004212200017
:101700001E004100810407000000EB000080FA0089
:10171000000006000A00FA00889FBE008A9FBE00F3
:10172000400798004E009000A00890004E009000E6
:1017300076004000750407004E009000B04890000D
:101740004E00900060019000F00190004E0090006B
:10175000204A90004E009000870B200080834300B9
:101760004E009000C5042000808242004E00900090
:101770002A082000000545004E009000F6054000B4
:101780004E009000000C9000900C90004E009000D5
:10179000680040008F87E800E1FF9F00829FBE0045
:1017A0008F87E800E4FF9F00050378008A02780035
:1017B0000B0278000801BE0041C0B30066FD0700BF
:1017C000E8875700200798002E0090000000E000F6
:1017D00064003A000000EB00100798000040EB00A6
:1017E000004F7800150037001E80FB00CE009000EF
:1017F0006012B0000100400090407800114798004E
:101800000A0037001E4090000080FB00E1006000ED
:101810001E00900001004000100798001E4090003C
:101820000080FB000000D100104798001E4090008F
:101830000004E000F3FF3A001E4FE8001E80FB00AA
:10184000CE009000A1109100810F5000E6FF3500FE
:1018500066004700740407000040EB00004F78006A
:101860003A0037001E009000CF80DE007DFB0700AD
:10187000800078004E009000A015B00023040700FF
:101880004E00900042122000000141004E009000E6
:10189000E40E2000000242004E009000A11520003E
:1018A000808040004E009000760040008201780069
:1018B00004017800E7FD07004E009000B04890005A
:1018C0004E00900060019000F00190004E009000EA
:1018D000204A90004E009000870B20008083430038
:1018E0004E009000C5042000808242004E0090000F
:1018F0002A082000000545004E009000F605400033
:101900004E009000000C9000900C90004E00900053
:10191000680040008F87E800E1FF9F00829FBE00C3
:101920008F87E800E4FF9F00050378008A027800B3
:101930000B0278000801BE0041C0B30006FD07009D
:10194000E8875700200798001E4FE8002E009000FF
:101950000000E00003003A006E4090009E4F10002F
:10196000C0FF39002E0090000000E00003003200AC
:101970004E009000AE009000310098002E009000C4
:101980004F05BE004F04BE000080FA0000000600B4
:101990000800FA00889FBE00200798002E009000E3
:1019A00010409000EE4F500004003A002E009000CE
:1019B00020489000604798000200370040C0B30004
:1019C00060479800EE409000214798002E0090005C
:1019D000760240002E009000200C90002E00900017
:1019E00000099000900990002E009000E80440004B
:1019F0008F87E8000040EB00E0FF9F006000B80028
:101A0000809FBE008F87E8002E409000E0FF9F007F
:101A10008003EB000003EB008002EB0088007800FD
:101A20000900780064FD0700E8875700000F780080
:101A30001E00E000030032002E0090009E0078009F
:101A4000310098001E0078004F04BE000080FA00AC
:101A5000000006000800FA00889FBE008A1F780078
:101A6000200798002E00900010409000F14F500089
:101A700004003A002E009000204890006047980033
:101A80000200370040C0B30060479800EE4090006D
:101A9000214798002E009000C4042000000242005C
:101AA0002E00900025082000808242002E00900029
:101AB000760440002E009000A00C90002E009000B4
:101AC00000099000900990002E00900068054000E9
:101AD0008F87E8000040EB00E0FF9F006000B80047
:101AE000809FBE008F87E8002E409000E0FF9F009F
:101AF0008003EB0004037800080278008900780076
:101B00000A0078002CFD0700E8875700000F7800D6
:101B10001E00E000030032002E0090009E007800BE
:101B2000310098001E0078004F0578004F04BE0079
:101B30000080FA00000006000600FA002007980066
:101B40000E80E800B8030700AE4090002E00900021
:101B500068004000EBFA0700000F78001E00E0006C
:101B6000030032002E0090009E00780031009800A3
:101B70001E0078000080FA00000006000600FA004F
:101B8000200798000000EB00000F78000E80E800AE
:101B9000A50307002E4090000004E000060032007C
:101BA0002E409000E14F5000030032005000200012
:101BB000000F7800190037002E00900010409000B0
:101BC000F34F50000B003A002E4090000004E0005C
:101BD00004003A00AE00900010C0B3009048980096
:101BE0000E003700AE009000D0C0B30090489800BF
:101BF0000A0037002E4090000004E00004003A0084
:101C0000AE00900010C0B300A04898000300370059
:101C1000AE00900060C0B300A04898001E00E00035
:101C2000030032002E0090009E00780031009800E2
:101C30001E0078000080FA00000006000400FA0090
:101C4000100798000E007800770307001E40780008
:101C50000004E000FBFF3A009E0090000000EB0053
:101C6000B00098001E009000300090000080FA0044
:101C7000000006000800FA00300798003E009000BF
:101C80007600400011002000200307003E00900075
:101C900080589000514798003E0090007600400028
:101CA00011002000190307003E00900080589000AA
:101CB000414798003E00900076004000410020001F
:101CC000120307003E009000760040003D0207002E
:101CD000008FBE003E009000804890005E40900063
:101CE00080CF5000040032003E00900068004000A9
:101CF000DE40900083FA07001E00BE008C03070040
:101D00003E009000804890004E40900080CF5000F0
:101D1000040032003E00900068004000CE40900079
:101D200078FA07000000EB000080FA0000000600CF
:101D30000200FA00000F78001E0078001CFA07006D
:101D4000800078001E007800310098001E007800A6
:101D5000300090000000E00007003A009E0078008C
:101D6000688040008040EB0066FA07008000780041
:101D70001E007800310098001E00780030009000AE
:101D80000080FA00000006000200FA00000F780050
:101D90001E007800300090000000E0001E003A00B5
:101DA0001E007800104078000004E0001A003A009D
:101DB0001E00E8001C0307001E007800A000900031
:101DC0001000900061004000E08048001E01780093
:101DD00010019800210198001E007800104090002A
:101DE000F74F50000A003E001E007800104090009F
:101DF0000080FB0080004000408021000080400007
:101E0000900078001E0078000100010002003700F9
:101E10001E007800F0FC07001E00780030009000E3
:101E20000080FA00000006000200FA00000F7800AF
:101E30001E00780007FA07000080FA000000060084
:101E40009001FA000E007800B9FF07000200370089
:101E50000E007800CCFF07003E0090000000E0007C
:101E600003003A001E4078000004E000F8FF320052
:101E70000E007800ECFF07003E0090000080FA00A2
:101E8000000006000200FA00BF0007003C18A8008E
:101E900000003700570307003AF8B7003AD8BF00F0
:101EA0000080FB00000F78001E007800E20F500059
:101EB0000A0032001E007800E30F50003D0032009F
:101EC0001E007800E10F500001003200F1FF3700E2
:101ED0007A00070040000700EEFF37007700070098
:101EE000470107003C00070020C0B3007C0007004A
:101EF00000C0EB006401070000C0EB0062010700B6
:101F00003500070030C0B300750007000000EB008B
:101F1000C0C1880007003700C0C180000000E80091
:101F2000C0C18800C1C18000900F2000808F500088
:101F300003003600210107000004E000F6FF320034
:101F4000250007005D0007002300070030C0B30034
:101F500063000700C0C180004200DD002E030700BF
:101F60000040EB003BF8B7000B003700DD00070036
:101F700029030700DB00070027030700D90007003B
:101F800025030700D7000700230307003BD8BF0045
:101F90000040E8003BF8B7003BD8BF008080FB0062
:101FA000C0C18000808F5000F0FF39000A00070098
:101FB000B8FF37002D010700590107007A0107001B
:101FC000660207009EFF0700C0C18800C0C18000F4
:101FD00011030700AFFF37000200FA0034D8BF003A
:101FE0000080FB00000F78001E007800E10F500019
:101FF000300032001E007800E10F500004003C0069
:102000001E0078000000E0000800320029003700C0
:102010001E007800E20F50000A0032001E00780017
:10202000E30F50001B003200220037005E01070062
:1020300010C0B3001401070010C0B30034F8B7009B
:102040001C00370035D8BF00E14F500008003A00AF
:1020500036D8BF00E14F500002003A00E800070008
:1020600001003700010107000040EB0035F8B70020
:102070003201070020C0B300030107004A01070036
:1020800010C0B3000001070010C0B30034F8B7005F
:10209000080037002901070020C0B300FA0007003C
:1020A0004101070010C0B300F700070010C0B300E3
:1020B00034F8B7000080FA00000006000000FA00C3
:1020C0001E010700A0C0B300EF00070036010700A3
:1020D0000040EB0034F8B7000080FA000000060072
:1020E0000400FA00004F78001E80FB0010079800E3
:1020F0001E009000E10F5000210032001E009000F1
:10210000E10F500004003C001E0090000000E000C1
:10211000080032001A0037001E009000E20F500045
:102120000F0032001E009000E30F50000300320049
:1021300013003700E1FF070011003700FF00070020
:1021400010C0B300D00007001701070020C0B30083
:10215000CD00070030C0B30034F8B70008003700E6
:10216000F600070020C0B300C70007000E010700FB
:1021700020C0B300C400070020C0B30034F8B7008B
:102180000080FA00000006000000FA00C8E2A80083
:10219000C902A900C922A900C8C2A900CAE2A900AF
:1021A000CB02A900CB22A900CAC2A9000080FA0074
:1021B000000006000800FA0040479800D800070019
:1021C00035D8BF00E14F500004003A0036D8BF00B8
:1021D000690007000040EB0035F8B70010C0B300FD
:1021E000004F78000040EB00304798003400370083
:1021F0004E4090001E4060000004E00002003A00E3
:102200009A000700010037007D000700AB000700BF
:10221000CAC2BF000080FB004700DE0020479800D4
:102220004E4090000080FB000000D1004047980025
:102230001E4090000080FB000000D1001047980075
:102240002E409000E14F500004003A001E409000E4
:1022500001C8B3000140400010479800B0000700DB
:1022600034D8BF00E24F500012003A003E409000C8
:10227000E64F50000F003A0010C0B30035F8B70029
:102280004E4090001E4060000004E00003003A0051
:102290000040EB0036F8B7000200370010C0B30072
:1022A00036F8B7001E4090000080FB003007980011
:1022B000090037003E4090000040E8003047980099
:1022C0003E409000E74F5000C9FF36001E4090008E
:1022D0000080FB00300798003E0090000080FA006C
:1022E000000006000400FA008D00070035D8BF008A
:1022F000E14F500004003A0036D8BF001E0007002E
:102300000040EB0035F8B7000040EB002047980094
:102310001300370069000700CAC2BF000080FB003D
:102320004700DE00104798001E80FB000000D1002F
:10233000004F78001E4090000004E00004003200CE
:102340001E40780001C8B30001404000004F7800F3
:10235000730007002E4090000040E80020479800DE
:102360002E409000E74F5000EAFF36001E80FB0031
:102370000080FA00000006000400FA0020479800E0
:102380002E4090000004E00002003A0037000700F1
:10239000010037001A00070048000700CAC2BF004A
:1023A0000080FB004700DE00004F78005C00070063
:1023B0001E80FB000080FA00000006000200FA0008
:1023C0003E000700CAC2BF000080FB004700DE00DD
:1023D000004F7800520007001E80FB000080FA00CA
:1023E000000006000000FA00CAC2BF000080FB0027
:1023F0004700DE000080FB000080FA0000000600BD
:102400000000FA003CD8BF006140600000C0EA0054
:10241000614060006140600000414000912C20005C
:1024200091407800D0CFB30000C06000024070003F
:10243000C9E2B7003CD8BF00614060006140600065
:1024400000414000B12C200091407800D0CFB30073
:1024500000C0600002407000CBE2B70040C1B30092
:10246000290207000080FA00000006000000FA00C0
:10247000CB22A900C922A90040C1B3002202070053
:102480000080FA00000006000400FA0020479800CF
:102490000040EB00004F7800030037000700070002
:1024A0001F0007001E4FE8002E4090009E4F1000B6
:1024B000FAFF39000080FA00000006000000FA0070
:1024C0003CD8BF006140600000C0EA00614060008D
:1024D00061416000912C200091407800E0CFB30072
:1024E00000C0600002407000C9E2B7003CD8BF00E5
:1024F0006140600061416000B12C20009140780093
:10250000E0CFB30000C0600002407000CBE2B70033
:1025100040C6B300FC0107000080FA00000006007E
:102520000000FA00CB02A900C902A90040C6B3000E
:10253000F50107000080FA00000006000000FA0024
:102540003CD8BF006140600000C0EA00614060000C
:10255000614060004601DD00812C20009140780040
:10256000F0CBB30000C0600002407000C8E2B700CA
:102570003CD8BF0061406000614060004601DD0062
:10258000A12C200091407800F0CBB30000C0600087
:1025900002407000CAE2B70040C1B300DA01070090
:1025A0000080FA00000006000000FA00CAC2A9007C
:1025B000C8C2A90040C1B300D30107000080FA00DF
:1025C000000006000800FA00300798006000B8001C
:1025D00010079800210798000000EB00000F78001A
:1025E000160037001E009000AE009000C808DD0005
:1025F0000080FD00804078000040EB00100798004C
:10260000210798001E007800BE0090000080E800BE
:1026100001004000104078000081FB000300200012
:102620001E009000AE0090000200700083807000D9
:1026300010079800210798001E0FE8003E00900048
:10264000100078009E0F5000E6FF3C001E00900036
:10265000AE0090000080FA00000006000600FA00BC
:10266000000F780012079800230798009E0078005A
:1026700010002000800878001E0090008040780044
:102680001E007800214098000080FA00000006003B
:102690000E00FA0040079800510798006207980062
:1026A00010002000300798004E0090009000780045
:1026B00021079800200037002E009000CE009000E7
:1026C0000080E80001004000904078002147980019
:1026D0002E009000DE0090000080E8000100400025
:1026E00090407800114798006E0090000000E000D4
:1026F0000B0032002E009000EE0090000080E800F9
:1027000001004000104F78002E4090001E406000F5
:10271000204798001E4090001E406000104798001F
:10272000AE4090001E40900080CF5000020032006A
:102730000000EB00300798003E0090000000E00031
:10274000060032002E0090000000E90020079800EB
:102750002E009000E10F4000D7FF3A003E009000AD
:102760000080FA00000006000600FA00000F780062
:1027700011079800220798001E0090009E00780024
:102780000080E80001004000104078008080FB00DD
:102790002E009000670010000088DE0061006000DD
:1027A0000080FA00000006000A00FA0010079800F6
:1027B0002107980032079800430798003E009000D8
:1027C000E7001000100020000100DD00004F78003D
:1027D0002E0090009E0090000080E8000100400064
:1027E00010407800804078001E40780000C0EA0069
:1027F00000C06000104798004E0090000000E0000C
:10280000030032001E4090001E40700010479800E8
:102810002E0090009E0090000080E8000100400023
:102820009E409000014878000080FA0000000600F9
:102830001000FA005007980061079800720798008E
:102840006E009000900078005E0090000108780013
:102850000040EB00004F98006E009000100F7800D1
:10286000240037001E007800EE0090000080E80091
:1028700001004000104078000080FB002007980015
:102880001E007800FE0090000080E800010040007B
:10289000104078000080FB0010079800AE00900008
:1028A0001E009000808040000E4890000080FB00D9
:1028B00000804000300798000040EB00004F980077
:1028C000BE009000F00F2000808F50000200360004
:1028D00010C0B300004F98001E0178003E00900029
:1028E00080417800DE0090000280E8000100400096
:1028F000034878001E0FE9000080EB009E0F1000D7
:10290000D8FF3A000080FA00000006000600FA0036
:1029100010079800210798001E009000AE0090005C
:10292000010878001E009000008FE80006003700C4
:102930001E0078003C0007002E0090000000E90017
:10294000200798001E0FE8002E0090000000E00015
:10295000F7FF3A000080FA00000006000000FA00CD
:102960000000EB0000408800C922A900C902A900AC
:10297000C8E2A800C8C2A9000080FA000000060052
:102980000400FA00000F78001107980010002000E2
:102990009E0F10000A003A001E0090006140600087
:1029A000614060004601DD00A12C200091407800CC
:1029B000F0CBB30000C0600002407000CAE2B70074
:1029C000200020009E0F10000A003A001E00900018
:1029D000614060006140600000414000B12C200077
:1029E00091407800D0CFB30000C06000024070007A
:1029F000CBE2B7001E00E00009003A001E00900084
:102A00006140600061416000B12C2000914078007D
:102A1000E0CFB30000C0600002407000CBE2B7001E
:102A20000080FA00000006000600FA00881F780007
:102A300020079800004080000000E00026003A00D7
:102A400000C0EB007400070022C2BF0061406000BC
:102A50000004E000FCFF3200660007001047980009
:102A600064000700004F78001E4090000080FB00CB
:102A7000C800DD001E80FB00008070000040880060
:102A80000000EB00100798000D00370022C2BF00C5
:102A9000614060000004E000FCFF32001E04900072
:102AA000540007008040780040802000000044006F
:102AB000014878001E0090000000E8001007980010
:102AC000014080001E009000810F5000EFFF390090
:102AD0000000EB0010408800114080004080200082
:102AE00000804000904078002E009000014878005F
:102AF000104080000000E800104088000040800086
:102B00000000E900004088004F0478000080FA00CF
:102B1000000006000000FA00CAC2BF000080FB00EF
:102B20004700DE000080FB000080FA000000060085
:102B30000800FA0020079800310798006000B800EC
:102B4000008FBE000600370010C0B3006E00070003
:102B50001E00BE0061004000E0804800008FBE0003
:102B60001E01BE002E009000BE009000800F51009C
:102B7000818F5900F4FF35000080FA000000060044
:102B80000000FA00C922A800C902A800C8E2A800F3
:102B9000C8C2A800C942A800C222A900C022A90038
:102BA000CB62A900C962A900C002A900C202A900A3
:102BB0002D23A9002D43A9002D63A9002D83A90071
:102BC000013220009140780000CEB30000C07000B8
:102BD00020E3B7000000EB008019880020F02100FE
:102BE000201988000000EB00101988000080FA000E
:102BF000000006000000FA0022C2BF006140600031
:102C00000004E000FCFF3200301180000080FB0077
:102C10000080FA00000006000200FA00004F780071
:102C200023C2BF00624060000004E000FCFF3A00E5
:102C30001E00FB00201188000080FA000000060042
:102C40000000FA00416A20009140780000CEB300F5
:102C500000C060005040B300A4E6B700416C200003
:102C60009140780000CEB30000C060003040B30057
:102C7000C4E6B70020022000401188000000EB00ED
:102C8000001188002062A8000000EB0010118800ED
:102C900021E2A8002342A8008560A9000080FA0074
:102CA000000006000600FA00404798000040EB00D4
:102CB000204798000E0037000000EB00000F78005E
:102CC00005003700A0CFB3000F0007001E007800FA
:102CD0000000E800000F78001E007800E30F5000AD
:102CE000F8FF36002E4090000040E8002047980092
:102CF000AE4090004E40900080CF5000EEFF390073
:102D00000080FA00000006000400FA002047980046
:102D10000040EB00004F7800130037000000000077
:102D200000000000000000000000000000000000A3
:102D30000000000000000000000000000000000093
:102D40000000000000000000000000000000000083
:102D50000000000000000000000000001E4078009D
:102D60000040E800004F78009E4078002E40900020
:102D700080CF5000E9FF39000080FA000000060013
:102D8000341800000A0000000000000004180000D1
:102D90003000000002000000FE080E0009220900B9
:102DA000200A8E000AEC0800EC08AC000ABC0A00FD
:102DB000000B6C000B8A0B00C80CC8000CC80C0080
:102DC0002A0D2A000D2A0D009C0DBE000DBE0D001F
:102DD000A0091E000E3A0E000008000004100000BA
:102DE00000000000000000000000FA004507A900F4
:102DF0000080EB00601988004227A90060FF0700EF
:102E00008FFF0700C002A900C202A8001DFC070036
:102E1000FFFF37000000FE00FFFFFF00FFFFFF0085
:102E2000FFFFFF00FFFFFF00FFFFFF00FFFFFF00AE
:102E3000FFFFFF00FFFFFF00FFFFFF00FFFFFF009E
:102E4000FFFFFF00FFFFFF00FFFFFF00FFFFFF008E
:102E5000FFFFFF00FFFFFF00FFFFFF00FFFFFF007E
:020000040001F9
:00000001FF
